:020000040000FA
:10000000012803138316033085000030860000307A
:10001000870083128316FC309F008312C1309F003B
:100020000511851264003E204420CF01CE01CC0A88
:100030004A204F085B208700071205150F21051184
:100040004E085B20870085160F218512FF30870040
:1000500041204420CF01CE01CC0A4A204F08A920DC
:100060008600861305150F2105114E08A92086006C
:1000700085160F218512FF30860012289F110F214F
:1000800008009F150F2108001F151F1945281E087D
:10009000CC0008006400CC0B4E280800CE0ACE1815
:1000A000CE1D5428CF0ACE01CF18CF1D4A280F30BD
:1000B000CE00CF000800CD004D1862285F28CD1873
:1000C0006B286528CD186E2868284D197D28712861
:1000D0004D19802874284D19832877284D198628B2
:1000E0007A28CD1999288928CD199B288B28CD19D4
:1000F0009D288D28CD199F288F28CD19A1289128BA
:10010000CD19A3289328CD19A5289528CD19A7285E
:10011000972811300800BD300800583008003830EA
:100120000800B63008003230080012300800B9303C
:1001300008001030080030300800FE300800FE30A3
:100140000800FE300800FE300800FE300800FE30D7
:100150000800CD004D18B028AD28CD18B928B32817
:10016000CD18BC28B6284D19CB28BF284D19CE284C
:10017000C2284D19D128C5284D19D428C828CD1911
:10018000E728D728CD19E928D928CD19EB28DB286D
:10019000CD19ED28DD28CD19EF28DF28CD19F1285C
:1001A000E128CD19F328E328CD19F528E52890306A
:1001B0000800D7300800A4300800C4300800CB3055
:1001C0000800C830080088300800D53008008030AA
:1001D0000800C0300800EF300800EF300800EF30B2
:1001E0000800EF300800EF300800EF30080014304E
:1001F000C2006430C1006430C0006400C00BFE283F
:10020000C10BFB28C20BF92808006430C100C830BC
:10021000C000C00B0929C10B072964000800643025
:10022000C000C00B1129640008000A30C000C00BD8
:060230001729640008001C
:02400E00BF3FB2
:00000001FF
